:0200000480007A
:100000006F00000B1300000013000000130000003D
:100010001300000013000000130000001300000094
:10002000232E11FE232C51FE232A61FE232871FE6C
:100030002326A1FE2324B1FE2322C1FE2320D1FECC
:10004000232EE1FC232CF1FC232A01FD232811FDA2
:100050002326C1FD2324D1FD2322E1FD2320F1FD30
:10006000130101FCEF00400B8320C10383228103B5
:1000700003234103832301030325C1028325810256
:1000800003264102832601020327C1018327810140
:100090000328410183280101032EC100832E810022
:1000A000032F4100832F010013010104730020304E
:1000B00097410000938181C11761000013018143C2
:1000C0001385C18197650000938585026308B5009B
:1000D00023200500130545006FF05FFF1735000072
:1000E0001305853E1301C1FF973500009385C53D7B
:1000F000630EB50083260500130545002320A100EB
:10010000E7800600032501006FF01FFE1301410088
:08011000EF20903D6F0000009C
:100118006780000003C75183930710046304F70046
:10012800678000008327050003A7C1839387970092
:10013800B387E7402320F5006780000003A64184C9
:1001480063080600032706002320E50003A6418470
:1001580083A5C1831306C6001305A0006F00100F06
:10016800130101FF2320210183A741842324810057
:100178000324050003A707002322910083AE47004C
:1001880003AE870003A3070183A8470103A88701DB
:1001980083A5070203A6470283A687022326110028
:1001A8009304050003A5C70183A7C7022320E40021
:1001B80003A70400232EA4002326F4022322D4013B
:1001C800930750002324C40123286400232A140120
:1001D800232C04012320B4022322C4022324D402A2
:1001E80023A6F4002326F4002320E40013050400CA
:1001F800EFF0DFF4832744006380070883A7040037
:100208008320C1000324810083AF070003AF4700A8
:1002180083AE870003AEC70003A3070183A8470185
:1002280003A8870183A5C70103A6070283A647027F
:1002380003A7870283A7C70223A0F40123A2E4012E
:1002480023A4D40123A6C40123A8640023AA14016B
:1002580023AC040123AEB40023A0C40223A2D40219
:1002680023A4E40223A6F402032901008324410005
:10027800130101016780000003A584009307600053
:10028800930584002326F400EF00500C83A74184D3
:100298000325C4001306C40083A707008320C100F8
:1002A800832441002320F400032481000329010052
:1002B8009305A000130101016F00407983C75183A2
:1002C80083A681839387F7FB93B71700B3E7D7001B
:1002D80023ACF18213072004238AE182678000009F
:1002E80013071004A38AE18223AC0182678000000F
:1002F800130101F613050003232E1108232C81088E
:10030800232A91072326B107232A910823282109A4
:100318002326310923244109232251092320610975
:10032800232E7107232C81072328A107EF00D0195A
:1003380023A0A18413050003EF00101983A70184EB
:1003480023A2A1842320F500930720002324F5008D
:10035800B7350080930780022326F5001306F001C5
:100368009385C5D02322050013050501EF00502F02
:100378003737008093074727032E472703A34700F3
:1003880083A8870003A8C70083A5070103A6470120
:1003980083A6870103D7C70183C7E701B73D00805C
:1003A800231EE102230FF1021387CD5D9307A000FE
:1003B8001305A000232EF7642320C1032322610222
:1003C80023241103232601032328B102232AC1026F
:1003D800232CD102EF005027373500801305C5D2F2
:1003E800EF0050221305A000EF00102683A7018319
:1003F800638A0760373500801305C5D5EF00902064
:100408001305A000EF00502437350080130585DB65
:10041800EF00100E1305A000EF0010233735008001
:100428009305800C130505DFEF00900CEF00902278
:100438003734008083274429373D0080032C4D2B17
:100448002326F10023A6A18293091000130444294E
:1004580093042000EFF0DFE8EFF05FE68347E40164
:1004680003264401032E4400032384008328C40088
:1004780003280401832684010357C401832EC10085
:10048800230FF104930501049307100013050102DB
:10049800232AC104232EF100232A91002320D10509
:1004A8002322C105232461042326110523280105DD
:1004B800232CD104231EE104EF00806203264101AE
:1004C8001335150023ACA18263CAC4029317260012
:1004D800B387C7009387D7FF13050600930530003D
:1004E80013068101232CF100EF0040560326410139
:1004F80013061600232AC100E3DAC4FC832681010F
:100508001385C1849385CD5DEF00405503A54184D3
:10051800930A1004130A3000EFF09FC403C7418305
:1005280093070004130B4D2B63F4E70213850A00AD
:1005380093053004EF00C0588327C10113871A00C0
:10054800630CF54483C74183937AF70FE3F057FFB1
:1005580083274101032B810113054101330AFA0264
:1005680093891900B34A6A03232A5101EFF09FBA0D
:100578009307900CE390F9EEEF00D00D23A4A1822D
:1005880037350080130505E2EF00D0071305A000FA
:10059800EF00900B37350080130505E3EF00900658
:1005A8001305A000EF00500A83A5C18337350080EA
:1005B800130585E637340080EF00807393055000FB
:1005C800130544E8EF00C07283A5818337350080A6
:1005D800130505EAEF00C07193051000130544E800
:1005E800EF00007183C55183373500801305C5EBD3
:1005F800EF000070B734008093051004138584ED74
:10060800EF00006F83C5418337350080130545EF40
:10061800EF00006E93052004138584EDEF00406D14
:100628009387C18483A5070237350080130505F138
:10063800EF00006C93057000130544E8EF00406B71
:10064800B73700809387C75D83A5C76537350080B6
:100658001305C5F2EF00C06937350080130585F42E
:10066800EF00407A37350080130545F7EF008079B1
:1006780003A74184B7370080138507F8832507004F
:100688002326F100373D0080EF0080663735008073
:100698001305C5F9EF00007703A741841305CDFCC6
:1006A800373C008083254700B73B0080B73900807E
:1006B800EF00006493050000130544E8EF00406371
:1006C80003A7418413058CFE3739008083258700F2
:1006D800330A6A41EF00C06193052000130544E81E
:1006E800EF00006103A7418413854B008325C700F1
:1006F800EF00006093051001130544E8EF00405F28
:1007080083A541841385090293850501EF00405EA6
:100718001305C903EF00006F37350080130505077F
:10072800EF00406E03A701848327C10083250700DB
:10073800138507F8EF00C05B3735008013050508FF
:10074800EF00406C83A701841305CDFC83A5470007
:10075800EF00005A93050000130544E8EF004059E4
:1007680083A7018413058CFE83A58700EF004058FA
:1007780093051000130544E8EF00805783A7018410
:1007880013854B0083A5C700EF0080569305200111
:10079800130544E8EF00C05583A5018413850902B9
:1007A80093850501EF00C0541305C903EF00806568
:1007B80083254101373500801305050CEF004053B0
:1007C80093055000130544E8EF00805293173A0050
:1007D800338A474137350080B3055A411305C50DA3
:1007E800EF0000519305D000130544E8EF00405096
:1007F80083258101373500801305850FEF00404FB1
:1008080093057000130544E8EF00804E8325C1016D
:100818003735008013054511EF00804D9305100012
:10082800130544E8EF00C04C3735008093050102FA
:1008380013050513EF00C04B373500801305C514A9
:10084800EF00405C37350080930501041305051857
:10085800EF00004A373500801305C519EF00805AAC
:100868001305A000EF00405E03A7C18283A5818223
:100878009307301FB385E54023A2B18263D0B71A2E
:100888003735008013058522EF00804603A5418295
:10089800EF20C00313040500EF208015B737008050
:1008A80003A6874C83A6C74CEF00D06FB7370080EC
:1008B80003A6074D83A6474DEF00D000EF20002484
:1008C80023A0A182B737008003A5874D93050400B4
:1008D800EF10004B23AEA180373500801305C523E8
:1008E800EF00004103A54182EF10507EB73700802A
:1008F8009305050003A5C74DEF10804813040500B4
:10090800EF10D07593040500EF10507C9305050097
:1009180013050400EF10102DB737008083A5074E8C
:10092800EF10007AEF10907313040500373500803C
:10093800938504001305C526EF00803B93079000BC
:1009480063D0871037350080930504001305052709
:10095800EF00003A1305A000EF00004F8320C10903
:100968000324810983244109032901098329C10832
:10097800032A8108832A4108032B0108832BC10716
:10098800032C8107832C4107032D0107832DC10602
:100998001301010A678000009305C10113050000D7
:1009A800EF00C01A03234B0083288B000328CB00D9
:1009B80003250B0183254B0103268B018356CB01AD
:1009C8000347EB0183C74183938A1A0023208105DB
:1009D8002322610423241105232601052328A104C9
:1009E800232AB104232CC104231ED104230FE104BC
:1009F80023AE318393FAFA0F138A0900E3F857B349
:100A08006FF01FB537350080130585D8EF00803F9C
:100A18001305A000EF0040436FF01F9F373500809B
:100A28001305051DEF00003E3735008013058520AE
:100A3800EF00403D1305A000EF0000416FF01FF2EA
:100A480013050003EF0040406FF0DFEF13052500AA
:100A5800B305B5002320B6006780000013075600D1
:100A68001308800C33080703131626009317270072
:100A78003305F5002320D500232CE5062322D500D5
:100A8800B307C800B387F50083A6070123AAE700C8
:100A980023ACE7001387160023A8E7008327050087
:100AA800B3850501B385C50037160000B305B60048
:100AB80023AAF5FA1307500023AEE18267800000ED
:100AC8001375F50F93F5F50F6306B50013050000D0
:100AD80067800000A38AA1821305100067800000C8
:100AE800130101FF232481002322910023261100F2
:100AF800130405009384050083C5340003452400CE
:100B0800EFF01FFCE31A05FE9385040013050400AB
:100B1800EF008043930700006358A0001307A0006C
:100B280023AEE182930710008320C10003248100D3
:100B38008324410013850700130101016780000029
:100B48001305E5FF1335150067800000130101FF49
:100B58002324810023229100232611001304050079
:100B680093840500EFF0DFFD630E050223A08400E7
:100B7800930710006300F4046304040413072000BF
:100B8800630CE404930740006314F40023A0E4001A
:100B98008320C10003248100832441001301010143
:100BA800678000009307300023A0F400930710002B
:100BB800E314F4FC03A7C1839307400663DAE70252
:100BC8008320C1000324810023A004008324410062
:100BD80013010101678000008320C1000324810004
:100BE80023A0F40083244100130101016780000061
:100BF8008320C100032481009307300023A0F40060
:100C0800832441001301010167800000130101FFE3
:100C18002324810023261100130405000345050041
:100C2800630A050013041400EF00002203450400C2
:100C3800E31A05FE8320C10003248100130101018A
:100C4800678000006F004020130101FD23229102FC
:100C58002326110223248102232021039304050063
:100C6800634C050413090100130409001307A000CD
:100C780063940400631E2401B3E7E4021304140020
:100C880093870703B3C4E402A30FF4FE6FF05FFE7B
:100C98001304F4FF03450400EFF0DFFAE31A24FF1E
:100CA8008320C10203248102832441020329010213
:100CB80013010103678000001305D002EFF09FF8CD
:100CC800B30490406FF01FFA03A78184B307A7000D
:100CD8003765008023A4F1841305C5CE9306004030
:100CE8003305E50063D4F600730010006780000048
:100CF800130101FB232C4101232611022324810225
:100D08002322910223202103232E3101232A51017A
:100D1800130A0500034505002322F1049307410344
:100D2800232AB102232CC102232ED1022320E1045D
:100D380023240105232611052326F1006308050253
:100D480013040000930A5002930430061309300775
:100D580093094006630E5503EFF0DFEE1304140009
:100D6800B3078A0003C50700E31605FE8320C10206
:100D78000324810283244102032901028329C1013A
:100D8800032A8101832A41011301010567800000BC
:100D9800930614003307DA006F000001638C270301
:100DA8006386370593861600834707001384060079
:100DB80013071700E38407FAE39297FE8327C1001D
:100DC80003A50700938747002326F100EFF09FE76C
:100DD8006FF0DFF88327C10003A50700938747005A
:100DE8002326F100EFF09FE26FF05FF78327C10041
:100DF80003A50700938747002326F100EFF0DFE4FF
:100E08006FF0DFF5130101FF232481002326110071
:100E18001304050003450500630A050013041400C4
:100E2800EF00800203450400E31A05FE1305A00045
:100E3800EF0080018320C100032481001305000016
:100E48001301010167800000B70710F023A0A7F085
:100E580067800000B70710F003A507F1678000005E
:100E6800B3C7A50093F737003307C500639607009B
:100E78009307300063E4C70293070500636CE5003D
:100E88006780000083C605009387170093851500C7
:100E9800A38FD7FEE3E8E7FE67800000937735006D
:100EA80063920708930705009376C7FF138606FE2B
:100EB80063F6C70883A3050083A2450083AF8500B6
:100EC80003AFC50083AE050103AE450103A3850149
:100ED80083A8C501938545029387470203A8C5FFE8
:100EE80023AE77FC23A057FE23A2F7FF23A4E7FF36
:100EF80023A6D7FF23A8C7FF23AA67FE23AC17FFA3
:100F080023AE07FF6FF0DFFA83C60500938717004B
:100F180093851500A38FD7FE93F63700E39606FE58
:100F28006FF09FF8930705006FF01FFF03A60500F9
:100F3800938747009385450023AEC7FEE3E8D7FEB5
:100F4800E3EAE7F4678000003367B5009303F0FF36
:100F58001377370063100710B7877F7F9387F7F7FA
:100F68000326050083A60500B372F6003363F60076
:100F7800B382F200B3E26200639272106316D6087D
:100F88000326450083A64500B372F6003363F600D6
:100F9800B382F200B3E26200639E720C6316D60657
:100FA8000326850083A68500B372F6003363F60036
:100FB800B382F200B3E262006398720C6316D6043F
:100FC8000326C50083A6C500B372F6003363F60096
:100FD800B382F200B3E262006392720C6316D60227
:100FE8000326050183A60501B372F6003363F600F4
:100FF800B382F200B3E26200639C720A13054501F2
:1010080093854501E30ED6F413170601939706015D
:10101800631EF7001357060193D706013305F740FF
:101028009375F50F63900502678000001357070159
:1010380093D707013305F7409375F50F63940500BF
:10104800678000001377F70F93F7F70F3305F74022
:10105800678000000346050083C6050013051500D8
:10106800938515006314D600E31606FE3305D640B3
:10107800678000001305450093854500E31CD6FCF6
:10108800130500006780000013058500938585001F
:10109800E312D6FC13050000678000001305C500A5
:1010A8009385C500E318D6FA130500006780000091
:1010B8001305050193850501E31ED6F81305000005
:1010C80067800000130101FD23248102232291027D
:1010D8002328610113040500130B0500B704100051
:1010E80013D5450123202103232E31012326710125
:1010F8009384F4FF23261102232C4101232A510152
:101108001375F57F930B060093890600B3F4B400BA
:1011180013D9F5016306050A9307F07F6306F510F6
:1011280093943400B7068000B3E4D400935ADB01EB
:10113800B3EA9A0013143B00130A15C0130B0000FE
:1011480013D54901B70410009384F4FF1375F57F94
:10115800B3F43401938F0B0093D9F901630205109E
:101168009307F07F6302F516B70780009394340065
:10117800B3E4F40093D7DB01B3E79700939F3B00F8
:10118800130515C01307000093162B00B3E6E600FD
:101198009386F6FF9305E000334639013305AA40EC
:1011A80063E0D5169725000093858512939626004F
:1011B800B386B60083A60600B386B600678006002D
:1011C800B3EA6401638E0A0663800404138504008D
:1011D800EF10502C930755FF1307C001634EF70219
:1011E800930AD001130485FFB38AFA40B3948400AC
:1011F800B35A5B01B3EA9A0033148B00130AD0C0C8
:10120800330AAA406FF09FF313050B00EF109028E4
:10121800130505026FF01FFC930485FDB31A9B00AC
:10122800130400006FF09FFDB3EA640163820A02B1
:10123800938A0400130AF07F130B30006FF05FF0FD
:1012480013040000130A0000130B10006FF05FEF87
:1012580013040000130AF07F130B20006FF05FEEF9
:10126800B3E77401638E07066380040413850400E2
:10127800EF105022130755FF9307C00163CEE70212
:101288009307D001930F85FFB387E740B394F40128
:10129800B3D7FB00B3E79700B39FFB011306D0C099
:1012A8003305A6406FF01FEE13850B00EF10901E5C
:1012B800130505026FF01FFC930785FDB397FB002C
:1012C800930F00006FF09FFDB3E77401638207027C
:1012D800938704001305F07F130730006FF0DFEAEF
:1012E800930F000013050000130710006FF0DFE9EB
:1012F800930F00001305F07F130720006FF0DFE85D
:1013080063E657016390FA36636EF4359395FA01F4
:10131800935614001317F40193DA1A0033E4D50036
:101328009397870013D88F013368F800935E0801FC
:10133800B3D5DA03131E0801135E0E019356040198
:1013480093988F00B3F4DA03938F0500B307BE02B6
:1013580093940401B3E6960063FEF600B386060193
:10136800938FF5FF63E8060163F6F600938FE5FFB8
:10137800B3860601B386F64033D3D60313140401AB
:1013880013540401B3F6D60393070300B3056E02A2
:1013980093960601B366D40063FEB600B3860601D1
:1013A8009307F3FF63E8060163F6B6009307E3FFCC
:1013B800B38606013384B640939F0F01B705010039
:1013C800B3EFFF001383F5FF93D60F01B3F76F0058
:1013D80013DF080133F36800B3836702B38466023E
:1013E800B307FF02B382E603B386970093D70301DE
:1013F800B387D70063F49700B382B20093D607018E
:10140800B3865600B70201009382F2FFB3F5570086
:1014180093950501B3F35300B38575006368D40051
:1014280093870F006314D4046372B704330717015A
:10143800B3321701B3820201330454009387FFFFCC
:101448006366880063148802636217036366D400C6
:10145800639E8600637CB700330717019387EFFF0D
:10146800B33F1701B38F0F013304F401B305B7403D
:101478003304D4403337B7003304E440930FF0FF0C
:1014880063048812B352D40393D605013374D4038A
:1014980013870200B30F5E021314040133E48600BD
:1014A800637EF401330404011387F2FF63680401C7
:1014B8006376F4011387E2FF330404013304F44133
:1014C800B356D4039395050193D505013374D4031A
:1014D800330EDE021314040133E4850093850600FD
:1014E800637EC401330404019385F6FF6368040135
:1014F8006376C4019385E6FF3304040113170701DB
:10150800B365B70013970501135707013304C441A6
:1015180013DE0501B30E670233036E02330ECF03E9
:10152800330FEF0213D70E01330F6F003307E701B4
:1015380063766700B7060100330EDE001353070118
:101548003303C301370E0100130EFEFFB376C70144
:1015580093960601B3FECE01B386D6016368640094
:10156800938F0500631064046380060433048800C5
:10157800938FF5FF63640403636664006314640275
:1015880063F0D80213971800B3381701338808019D
:10159800938FE5FF33040401930807006314640084
:1015A8006384160193EF1F009306F53F635AD0102A
:1015B80013F77F006300070213F7FF00930540004D
:1015C800630AB70093854F00B3BFF501B387F701EE
:1015D800938F050013977700635A0700370700FFBA
:1015E8001307F7FFB3F7E700930605401307E07FFB
:1015F800634AD7181397D70193DF3F003367F70182
:1016080093D73700B70510009385F5FFB3F7B700F8
:10161800B70510809385F5FF93F6F67F93964601FC
:10162800B3F7B7008320C102032481021316F60121
:10163800B3E7D700B3E6C7008324410203290102B8
:101648008329C101032A8101832A4101032B010156
:10165800832BC100130507009385060013010103BE
:10166800678000001305F5FF130700006FF05FCBDC
:101678001306090093870A00930F040013070B0051
:10168800930620006300D710930630006302D70E3C
:1016980093061000E31AD7F0930700001307000021
:1016A8006F004009138609006FF09FFDB707080017
:1016B800930F000013060000130730006FF05FFC63
:1016C80093051000B385D54013078003E346B7FCA4
:1016D8001307F0016344B7061305E5413397A700E4
:1016E800B3D6BF003395AF003367D7003335A000BA
:1016F8003367A700B3D7B7009376770063800602F5
:101708009376F70093054000638AB6009306470076
:1017180033B7E600B387E700138706009396870080
:1017280063CA06069396D7011357370033E7E600D6
:1017380093D73700930600006FF0DFEC130710FE15
:101748003307D7401308000233D7E7009306000099
:10175800638605011305E543B396A70033E5F60153
:101768003335A0003367A700930700006FF0DFF858
:10177800B7070800130700009306F07F1306000060
:101788006FF05FE893070000130700009306F07FEF
:101798006FF05FE79307000013070000930610003F
:1017A8006FF05FE6130101FD23202103232A510175
:1017B8003709100093DA4501232E3101232C41010A
:1017C80023286101232671011309F9FF2326110239
:1017D800232481022322910293FAFA7F130B050036
:1017E800930B0600138A06003379B90093D9F501E3
:1017F80063880A0A9307F07F6386FA10370480002B
:1018080013193900336989001354D501336424014D
:1018180093143500938A1AC0130B000013554A011C
:10182800370910001309F9FF1375F57F337949015A
:1018380013870B00135AFA01630405109307F07F0E
:101848006304F516B7078000131939003369F900E6
:1018580093D7DB01B3E7270113973B00130515C0A6
:101868009306000093152B00B3E5D5003385AA0035
:101878009385F5FF9308E00033C649011308150066
:1018880063E0B81617250000130545A893952500B1
:10189800B385A50083A50500B385A500678005006D
:1018A8003364A900630E04066300090413050900E4
:1018B800EF10403E930755FF1307C001634CF70232
:1018C8001304D001930485FF3304F44033199900BD
:1018D80033548B0033642401B3149B00930AD0C0A3
:1018E800B38AAA406FF05FF3EF10C03A1305050200
:1018F8006FF05FFC130485FD33148B009304000024
:101908006FF0DFFD3364A90063040402930405004B
:1019180013040900930AF07F130B30006FF01FF0D7
:1019280093040000930A0000130B10006FF01FEFE0
:1019380093040000930AF07F130B20006FF01FEE52
:10194800B3677901638E070663000904130509006C
:10195800EF104034930655FF9307C00163CED702BA
:101968009307D001130785FFB387D7403319E900E0
:10197800B3D7FB00B3E727013397EB009306D0C03A
:101988003385A6406FF0DFED13850B00EF10803034
:10199800130505026FF01FFC930785FDB397FB0045
:1019A800130700006FF09FFDB36779016382070298
:1019B800930709001305F07F930630006FF09FEA44
:1019C8001307000013050000930610006FF09FE94D
:1019D800130700001305F07F930620006FF09FE8BF
:1019E800B70F0100138FFFFF93D6040113530701AC
:1019F800B3F4E4013377E701B3089302B305970220
:101A0800B382E602338E580093D80501B388C80123
:101A1800B38E660263F45800B38EFE0113D9080131
:101A2800B3F8E80193DF0701B3F5E501B3F3E70184
:101A380093980801B388B800B3877602B3859302F8
:101A4800B3849F02338EF40093D40501B384C40198
:101A5800B386F60363F6F400B7070100B386F60011
:101A680013DF0401B7090100330FDF009386F9FF84
:101A7800B3F4D400B3F5D50093570401939404014B
:101A88003374D400B384B400B306870233099900D1
:101A9800338EE702B30583023307F3023383C501AC
:101AA80093D50601B385650063F4C5013307370193
:101AB80013D30501B7090100B302E3001387F9FF47
:101AC800B3F5E500B3F6E600338383029395050189
:101AD800B385D5003387770233848F02338EFF02B4
:101AE8003304E40093570301338487006374E400EC
:101AF800330E3E01B70701009387F7FFB376F40072
:101B08003373F30093960601B38E2E01B3866600F5
:101B1800B3B49E00B386E601B3879600B38EBE00C9
:101B2800B3B5BE0033835700B30FB300B3B6E601B5
:101B3800B3B79700B3E7F6001354040133335300E7
:101B4800B3B5BF00B3878700B365B300B387B700E9
:101B5800B387C70113D77F0193979700B3E7E700CF
:101B680013979E00336717013337E00093DE7E0139
:101B780093969F003367D7013367D7009396770012
:101B880063DA0610935617001377170033E7E60059
:101B98009396F7013367D70093D717009305F83F5B
:101BA800635EB00E93767700638006029376F70043
:101BB80013054000638AA6009306470033B7E60082
:101BC800B387E700138706009396770063DA060069
:101BD800B70600FF9386F6FFB3F7D70093050840D2
:101BE8009306E07F63CEB616935637001397D70156
:101BF8003367D70093D73700B70610009386F6FFF0
:101C0800B3F7D70093F6F57FB70510809385F5FFF6
:101C180093964601B3F7B7008320C10203248102DB
:101C28001316F601B3E7D700B3E6C70083244102D1
:101C3800032901028329C101032A8101832A410161
:101C4800032B0101832BC1001305070093850600B0
:101C5800130101036780000013860900930704003D
:101C68001387040093060B0093052000638AB60EC1
:101C780093053000638CB60C93051000E390B6F220
:101C880093070000130700006F00800813060A007E
:101C98006FF09FFD130805006FF05FF0130510004B
:101CA8003305B54093068003E3CCA6FC9306F00108
:101CB80063C4A6061308E841B3960701B355A70005
:101CC80033170701B3E6B6003337E00033E7E60021
:101CD800B3D7A70093767700638006029376F70060
:101CE80093054000638AB6009306470033B7E600C1
:101CF800B387E700138706009396870063CA060632
:101D08009396D7011357370033E7E60093D7370088
:101D1800930500006FF05FEE930610FEB386B640A1
:101D280093080002B3D6D700930500006306150197
:101D38001308E843B395070133E7E5003337E000BC
:101D480033E7E600930700006FF0DFF8B7070800F5
:101D5800130700009305F07F130600006FF0DFE91A
:101D680093070000130700009305F07F6FF0DFE88A
:101D78009307000013070000930510006FF0DFE7DA
:101D8800130101FE232A9100232631019354750182
:101D9800B709800023282101232441019389F9FFF1
:101DA800232E1100232C81002322510193F4F40FD8
:101DB800138A0500B3F9A9001359F50163880408CB
:101DC8009307F00F6384F40A93993900B707000466
:101DD800B3E9F900938414F8930A000013557A01C3
:101DE800370480001304F4FF1375F50F33744401AE
:101DF800135AFA01630C05089307F00F6308F50AF4
:101E080013143400B70700043364F400130515F8FD
:101E18009307000093962A00B3E6F6009386F6FF30
:101E28001307E000334649013385A4406360D70AAD
:101E3800971500009385455193962600B386B60002
:101E480003A706003307B70067000700638A090283
:101E580013850900EF0010649307B5FF9304A0F8F9
:101E6800B399F900B384A4406FF01FF79304F00FFF
:101E7800930A2000E38409F6930A30006FF01FF6F6
:101E880093040000930A10006FF05FF5630A0402E0
:101E980013050400EF0010609307B5FF3314F40036
:101EA8009307A0F83385A7406FF09FF61305F00F4E
:101EB80093072000E30004F6930730006FF09FF5C6
:101EC80013050000930710006FF0DFF41318540097
:101ED80063F6890E1305F5FF9306000013540801F5
:101EE80033D38902B70701009387F7FFB377F80068
:101EF80093D6060133F7890293050300B388670276
:101F08001317070133E7E600637E1701330707015C
:101F18009305F3FF63680701637617019305E3FFF1
:101F28003307070133071741B3588702337787020E
:101F3800B3861703931707011387080063FED700BA
:101F4800B38707011387F8FF63E8070163F6D70033
:101F58001387E8FFB387070113940501B387D740B8
:101F68003364E400B337F0003364F4001307F50773
:101F78006350E00A93777400638A07009377F4004C
:101F8800930640006384D700130444009317440069
:101F980063DA0700B70700F89387F7FF3374F40094
:101FA800130705089307E00F1354340063D2E70CB6
:101FB800130400001307F00F6F00800B9396F901CC
:101FC80093D919006FF09FF11306090013840900D3
:101FD80093870A0013072000E38CE7FC13073000FF
:101FE8006382E70813071000E392E7F81304000080
:101FF800130700006F00C00713060A006FF09FFD6B
:102008003704400013060000930730006FF09FFC70
:1020180093071000B387E7401307B001E348F7FCC4
:102028001305E509B357F4003314A40033348000D2
:1020380033E4870093777400638A07009377F4008A
:10204800130740006384E700130444009317540007
:1020580013543400E3DE07F81304000013071000DC
:102068006F000001370440001307F00F130600004B
:10207800370580001305F5FF3374A4003705808009
:102088001305F5FF1377F70F3374A40013177701BF
:102098003364E4001315F6013365A4008320C101FD
:1020A8000324810183244101032901018329C100FB
:1020B800032A8100832A410013010102678000007E
:1020C800130101FE232A910023282101B70480006F
:1020D8001359750123263101232251019384F4FFFA
:1020E800232E1100232C8100232441011379F90F99
:1020F800938A0500B3F4A4009359F501630A09080B
:102108009307F00F6306F90A93943400B7070004A5
:10211800B3E4F400130919F8130A000013D57A017F
:10212800370480001304F4FF1375F50F337454015A
:1021380093DAFA01630E05089307F00F630AF50AAC
:1021480013143400B70700043364F400130515F8BA
:102158009306000093172A00B3E7D7003305A900B8
:102168009387F7FF1307E00033C6590113081500DA
:102178006360F70A171700001307C7209397270013
:10218800B387E70083A70700B387E70067800700E6
:10219800638A040213850400EF00D02F9307B5FF6C
:1021A8001309A0F8B394F4003309A9406FF0DFF6DF
:1021B8001309F00F130A2000E38204F6130A300013
:1021C8006FF0DFF513090000130A10006FF01FF518
:1021D800630A040213050400EF00D02B9307B5FF30
:1021E8003314F4009307A0F83385A7406FF05FF627
:1021F8001305F00F93062000E30E04F49306300055
:102208006FF05FF513050000930610006FF09FF460
:10221800B70701001383F7FF13D70401935604018E
:10222800B3F4640033746400B3888402B30587028E
:102238003304D702B386960293D40801B386B60056
:10224800B384D40063F4B4003304F400B3F7640037
:1022580093970701B3F86800B387170113976700CE
:1022680093D404013337E00093D7A7013384840063
:10227800B367F700131464003364F4009317440041
:1022880063DE070C935714001374140033E48700BB
:102298001307F8076358E00C93777400638A070004
:1022A8009377F400930640006384D7001304440036
:1022B8009317440063DA0700B70700F89387F7FF1E
:1022C8003374F400130708089307E00F63CCE70E94
:1022D800935734006F000003138609001384040029
:1022E80093060A0093072000638EF60C93073000CC
:1022F8006382F60C93051000930700001307000093
:10230800E398B6F8370480001304F4FF370580809B
:10231800B3F787001305F5FF8320C101032481016A
:102328001377F70FB3F7A700131777011315F60103
:10233800B3E7E70083244101032901018329C10090
:10234800032A8100832A410033E5A7001301010213
:102358006780000013860A006FF0DFF81308050095
:102368006FF01FF393071000B387E7401307B0011E
:102378006340F7061308E809B357F400331404015F
:102388003334800033E4870093777400638A07004E
:102398009377F400130740006384E70013044400B4
:1023A8009317540063CA07029357340013070000B9
:1023B8006FF05FF5B70740001307F00F1306000032
:1023C8006FF05FF4930700001307F00F6FF09FF3AF
:1023D800930700006FF09FFD93070000130710009C
:1023E8006FF05FF2B70780009387F7FF130101FFD3
:1023F80033F7A7009356750113D67501B3F7B700E5
:10240800232291002320210193F6F60F1318370099
:102418001376F60F23261100232481001307F00FEB
:102428009354F501138906001305060093D5F501A9
:10243800939737006314E6006394070093C515006B
:102448003387C640639A951A6356E00A63160606F0
:10245800639C07009307F00F638CF604930708004A
:10246800138506006F00C0141307F7FF631E0702E9
:10247800B38707011385060013975700635A07129D
:10248800130515001307F00F630EE5323707007EBA
:1024980093F617001307F7FF93D71700B3F7E70072
:1024A800B3E7D7006F00C0101306F00F639EC60095
:1024B800930708006F0040071306F00FE38AC6FE73
:1024C80037060004B3E7C7001306B0016356E600F9
:1024D800930710006FF0DFF9130600023306E64099
:1024E800B3D5E700B397C700B337F000B3E7F500FB
:1024F8006FF01FF863000708639C06026318080062
:102508001307F00F6316E60A6F0000029306F0FF48
:102518006316D700B38707016FF01FF69306F00F15
:102528001347F7FF6310D6021305F00F6F0040083A
:102538009306F00FE30AD6FEB70600043307E0401F
:102548003368D8009306B00163D6E600130710007D
:102558006F00C001930600023356E8003387E64057
:102568003317E8003337E0003367E600B387E70046
:102578006FF09FF0138516001376F50F1307100000
:102588006342C70663940604130500006302080249
:1025980063860722B387070113975700635A07001A
:1025A800370700FC1307F7FFB3F7E7001305100020
:1025B80013F77700630A072013F7F7009306400024
:1025C8006304D720938747006F000020E30E08F4C8
:1025D800E38007EEB70700021305F00F930400002D
:1025E8006F00801E1307F00F630EE51C3307F80019
:1025F800935717006FF0DFFB6350E008631606047B
:10260800E38A07E41307F7FF63140702B307F840E8
:102618001385060013975700E35C07F83704000496
:102628001304F4FF33F48700130905006F008013C7
:102638001306F00FE38EC6E61306B0016350E602F8
:10264800930710006FF09FFC1306F00FE382C6E6B5
:1026580037060004B3E7C7006FF01FFE1306000239
:10266800B3D5E7003307E640B397E700B337F00088
:10267800B3E7F5006FF09FF963020708639E06024F
:10268800631808001307F00F938405006FF09FE7A5
:102698009306F0FF6318D700B387074193840500BA
:1026A8006FF05FF79306F00F1347F7FF6310D6023A
:1026B800938405006FF05FE79306F00FE30AD6FEF8
:1026C800B70600043307E0403368D8009306B0012A
:1026D80063D6E600130710006F00C00193060002DE
:1026E8003356E8003387E6403317E8003337E00015
:1026F8003367E600B387E7406FF05FFA1387160089
:102708001377F70F130610006344E604639C060270
:102718006318080063980712130500006FF01FEC98
:10272800638607123307F84093165700B3870741AB
:1027380063CA061093070700631007069307000093
:102748006FF09FFDE31608E8E39407F66FF09FE843
:102758003304F840131754006354070433840741C3
:102768009384050013050400EF00C0521305B5FF5C
:102778003314A400634A25033305254113051500C6
:1027880013070002B357A4003305A7403314A4006D
:1027980033348000B3E78700130500006FF05FE172
:1027A800E30E04F86FF01FFCB70700FC9387F7FFF0
:1027B8003305A940B377F4006FF09FDF9307080053
:1027C8006FF01FDF9307000013975700635E070041
:1027D800130515001307F00F630EE506370700FC15
:1027E8001307F7FFB3F7E7001307F00F93D7370086
:1027F8006318E50063860700B707400093040000EC
:10280800370780001307F7FF1375F50FB3F7E700D5
:1028180013177501370580808320C10003248100C8
:102828001305F5FF33F5A7009394F4013365E5002C
:102838003365950003290100832441001301010138
:1028480067800000938405006FF01FF59307080068
:102858006FF09FF4930700006FF01FF937068000B0
:10286800135775019307F6FF1377F70F9305E007E2
:10287800B3F7A7009356F50163F6E5049305D0096D
:1028880063FAE500370500801345F5FF3385A60098
:102898006780000033E5C7009307500963DCE70051
:1028A8001307A7F63315E500638006023305A04039
:1028B80067800000930760093387E7403355E500D8
:1028C8006FF09FFE1305000067800000130101FFF1
:1028D800232611002324810023229100630205107E
:1028E800130405009354F501635405003304A04014
:1028F80013050400EF00003A9307E009B387A740E7
:10290800130760096340F706130780006356A700A2
:10291800130585FF3314A400370580001305F5FF60
:1029280093F7F70F3374A40013957701B7078080E6
:102938009387F7FF3374F400B70700803364A4006B
:1029480093C7F7FF1395F4013374F4003365A400BB
:102958008320C10003248100832441001301010165
:1029680067800000130790096350F70213075000AF
:102978003307A7409306B5013357E4003314D40056
:102988003334800033648700130750006356A70070
:102998001307B5FF3314E400370700FC1307F7FFEC
:1029A800937674003377E400638A06001374F400A6
:1029B800930640006304D40013074700931657009A
:1029C80063DC0600B70700FC9387F7FF3377F7004F
:1029D8009307F009B387A740135437006FF0DFF36C
:1029E8001304000093070000930400006FF0DFF267
:1029F80093577501130101FF93F7F70F2324810003
:102A08001387170037048000232291001304F4FF72
:102A1800232611001377F70F930610003374A400D0
:102A28009354F50163D2E6061385073893573400AB
:102A38001314D401370710001307F7FFB3F7E700A3
:102A4800370710801307F7FF1375F57F1315450136
:102A5800B3F7E70037070080B3E7A7001347F7FF8E
:102A68001395F401B3F7E70033E7A7008320C1000B
:102A78001305040003248100832441009305070003
:102A880013010101678000006394070463020406D0
:102A980013050400EF0000209307A00063C2A702FB
:102AA8009307B000B387A74013075501B357F40045
:102AB8003314E400130790383305A7406FF09FF7ED
:102AC800930755FFB317F400130400006FF09FFE3F
:102AD80093070000630A040093573400370708007F
:102AE8001314D401B3E7E7001305F07F6FF09FF4E8
:102AF80093070000130500006FF0DFF3370610009E
:102B08001306F6FF3376B60013D845019357D5015F
:102B18001378F87F1316360033E6C70093071800BA
:102B280093F7F77F9306100093D5F5011317350037
:102B380063D6F60A930608C89307E00F63C2D70C5A
:102B48006340D008930790FE63C4F612B70780006D
:102B58001305E0013366F6003305D5409307F0010D
:102B680063C8A702130828C8B3170701B337F000D2
:102B7800331606013355A700B3E7C700B367F5005E
:102B88009306000013F77700630007086F00C00E74
:102B98009307E0FFB386D74093070002B356D600E9
:102BA800930800006306F500130828CAB318060145
:102BB800B3E7E800B337F000B3E7F6006FF05FFC67
:102BC800131565003335A000131636009357D70147
:102BD8003366C500B367F6006FF0DFFAB367E60047
:102BE80063160800B337F0006FF09FF99306F00FF3
:102BF800638C070013163600B70700026FF09FFDBD
:102C0800930700009306F00F13975700635E0700C1
:102C1800938616001307F00F638AE606370700FC51
:102C28001307F7FFB3F7E7001307F00F93D7370041
:102C38006398E60063860700B70740009305000025
:102C4800370580001305F5FFB3F7A7003705808027
:102C58001305F5FF93F6F60F93967601B3F7A700E1
:102C68009395F501B3E7D70033E5B7006780000017
:102C7800930710009306000013F7F70013064000AF
:102C8800E304C7F8938747006FF01FF89307000025
:102C98006FF09FF9B7070100637AF5029307F00F09
:102CA800B3B7A70093973700130700023307F7401D
:102CB800B357F5001705000013058570B307F50035
:102CC80003C507003305A7406780000037070001E8
:102CD80093070001E36AE5FC930780016FF0DFFCCE
:102CE800130101FF23261100EFD08FE08320C100DC
:102CF800B70710F023A007F2130500001301010124
:042D080067800000E0
:102D0C004448525953544F4E452050524F4752410C
:102D1C004D2C20534F4D4520535452494E470000E3
:102D2C004468727973746F6E652042656E63686D6A
:102D3C0061726B2C2056657273696F6E20322E3166
:102D4C0020284C616E67756167653A204329000045
:102D5C0050726F6772616D20636F6D70696C656422
:102D6C0020776974682027726567697374657227A8
:102D7C0020617474726962757465000050726F67BB
:102D8C0072616D20636F6D70696C65642077697416
:102D9C00686F757420277265676973746572272074
:102DAC00617474726962757465000000506C6561C1
:102DBC007365206769766520746865206E756D6231
:102DCC006572206F662072756E73207468726F75F1
:102DDC006768207468652062656E63686D61726BEC
:102DEC003A200000457865637574696F6E207374C2
:102DFC00617274732C2025642072756E7320746854
:102E0C00726F756768204468727973746F6E650AA7
:102E1C0000000000457865637574696F6E20656EFF
:102E2C006473000046696E616C2076616C75657325
:102E3C00206F6620746865207661726961626C65CA
:102E4C0073207573656420696E20746865206265F3
:102E5C006E63686D61726B3A00000000496E745FBE
:102E6C00476C6F623A202020202020202020202038
:102E7C002025640A00000000202020202020202093
:102E8C0073686F756C642062653A20202025640A93
:102E9C0000000000426F6F6C5F476C6F623A20203D
:102EAC0020202020202020202025640A0000000063
:102EBC0043685F315F476C6F623A202020202020EE
:102ECC00202020202025630A000000002020202044
:102EDC002020202073686F756C642062653A202076
:102EEC002025630A0000000043685F325F476C6F67
:102EFC00623A202020202020202020202025630A38
:102F0C00000000004172725F315F476C6F625B388A
:102F1C005D3A2020202020202025640A000000009B
:102F2C004172725F325F476C6F625B385D5B375D1D
:102F3C003A2020202025640A0000000020202020B8
:102F4C002020202073686F756C642062653A202005
:102F5C00204E756D6265725F4F665F52756E7320A1
:102F6C002B203130000000005074725F476C6F6290
:102F7C002D3E000020205074725F436F6D703A201C
:102F8C0020202020202020202025640A0000000082
:102F9C00202020202020202073686F756C64206214
:102FAC00653A20202028696D706C656D656E7461C2
:102FBC0074696F6E2D646570656E64656E7429003E
:102FCC00202044697363723A202020202020202086
:102FDC00202020202025640A000000002020456EBF
:102FEC00756D5F436F6D703A2020202020202020CB
:102FFC002025640A000000002020496E745F436F96
:10300C006D703A2020202020202020202025640ACA
:10301C000000000020205374725F436F6D703A20E3
:10302C0020202020202020202025730A00000000D2
:10303C00202020202020202073686F756C64206273
:10304C00653A2020204448525953544F4E45205045
:10305C00524F4752414D2C20534F4D452053545203
:10306C00494E47004E6578745F5074725F476C6FC1
:10307C00622D3E00202020202020202073686F75B8
:10308C006C642062653A20202028696D706C656D37
:10309C00656E746174696F6E2D646570656E6465C0
:1030AC006E74292C2073616D652061732061626FD1
:1030BC0076650000496E745F315F4C6F633A202077
:1030CC0020202020202020202025640A0000000041
:1030DC00496E745F325F4C6F633A202020202020B1
:1030EC00202020202025640A00000000496E745F17
:1030FC00335F4C6F633A202020202020202020209A
:10310C002025640A00000000456E756D5F4C6F63EE
:10311C003A20202020202020202020202025640A56
:10312C00000000005374725F315F4C6F633A2020D3
:10313C0020202020202020202025730A00000000C1
:10314C00202020202020202073686F756C64206262
:10315C00653A2020204448525953544F4E45205034
:10316C00524F4752414D2C20312753542053545227
:10317C00494E47005374725F325F4C6F633A2020A4
:10318C0020202020202020202025730A0000000071
:10319C00202020202020202073686F756C64206212
:1031AC00653A2020204448525953544F4E452050E4
:1031BC00524F4752414D2C2032274E4420535452EB
:1031CC00494E47004D656173757265642074696D75
:1031DC006520746F6F20736D616C6C20746F206F41
:1031EC00627461696E206D65616E696E6766756C7F
:1031FC0020726573756C747300000000506C65610F
:10320C00736520696E637265617365206E756D629E
:10321C006572206F662072756E730000436C6F636D
:10322C006B206379636C65733D2564200A00000094
:10323C00444D49505320706572204D687A3A2020D5
:10324C002020202020202020202020202020202072
:10325C0020202020202020202020202000000000E2
:10326C0025642E00256400004448525953544F4E97
:10327C00452050524F4752414D2C2031275354205A
:10328C00535452494E4700004448525953544F4EE0
:10329C00452050524F4752414D2C2032274E44204E
:1032AC00535452494E4700004448525953544F4EC0
:1032BC00452050524F4752414D2C20332752442029
:1032CC00535452494E470000B8E4FFFFCCE3FFFFD4
:1032DC00D8E3FFFFCCE3FFFFA4E4FFFFCCE3FFFF49
:1032EC00D8E3FFFFB8E4FFFFB8E4FFFFA4E4FFFF5F
:1032FC00D8E3FFFFA4E3FFFFA4E3FFFFA4E3FFFF7A
:10330C00E0E3FFFF60E9FFFF60E9FFFF84E9FFFFF7
:10331C0054E9FFFF54E9FFFF44EAFFFF84E9FFFF94
:10332C0054E9FFFF44EAFFFF54E9FFFF84E9FFFF84
:10333C0050E9FFFF50E9FFFF50E9FFFF44EAFFFFB0
:10334C006CECFFFFA8ECFFFFB4ECFFFFA8ECFFFF59
:10335C0020EDFFFFA8ECFFFFB4ECFFFF6CECFFFFD0
:10336C006CECFFFF20EDFFFFB4ECFFFF84ECFFFFE4
:10337C0084ECFFFF84ECFFFFBCECFFFF64EFFFFF6E
:10338C0064EFFFFFD4EFFFFF5CEFFFFF5CEFFFFF8D
:10339C0034F0FFFFD4EFFFFF5CEFFFFF34F0FFFFD3
:1033AC005CEFFFFFD4EFFFFF58EFFFFF58EFFFFF7D
:1033BC0058EFFFFF34F0FFFF000102020303030389
:1033CC0004040404040404040505050505050505A9
:1033DC000505050505050505060606060606060689
:1033EC000606060606060606060606060606060671
:1033FC000606060606060606070707070707070759
:10340C000707070707070707070707070707070740
:10341C000707070707070707070707070707070730
:10342C000707070707070707070707070707070720
:10343C000707070707070707080808080808080808
:10344C0008080808080808080808080808080808F0
:10345C0008080808080808080808080808080808E0
:10346C0008080808080808080808080808080808D0
:10347C0008080808080808080808080808080808C0
:10348C0008080808080808080808080808080808B0
:10349C0008080808080808080808080808080808A0
:1034AC000808080808080808080808080808080890
:0834BC000808080808080808C8
:1034C8000000000080842E41000000205FA012420E
:0C34D800F90295503353DE470000C84253
:040000058000000077
:00000001FF
